:1000000083120313850105289028860107309F007D
:1000100083168E15B0308500F730860028308100B9
:100020000F3092008C14831295010F3097007C30B2
:100030009200E001E101E201E301F001F101F201CE
:10004000F301F401F501F601F701F801F901FA01F4
:10005000FB01FC01FD01FE01FF01061B342806081F
:10006000FF3AB739FB00612883163F309B001C1410
:100070001A08FB008312851E7014851FF014700887
:1000800003196128FE3E03194A2803184F288030BF
:10009000FB0653287B08BF39103EFB0053287B0822
:1000A000F739013EFB0083161C153F309B007B088F
:1000B000B7399A0055309D00AA309D009C141C1140
:1000C00083128316860183123C30FB1B3230E20020
:1000D00007307B05043E9500FB1A71287B1E88289B
:1000E00081287B1E7C287030FC000830FD007030B9
:1000F000FE000830FF0088280830FD000830FF00AF
:100100008828FC010F30FD007030FE000830FF0031
:100110008C10FF3081000B110B178B1700008E28FD
:100120008312851A9628F00F9728AE28F001851BB8
:100130009C28F10F9D28B428F1010B1DBA280B1142
:10014000FF308100F20A62087206031DBA28F2012C
:10015000F30A3C307306031DBA28F301F40A3C305D
:100160007406031DBA28F401F50A18307506031D3C
:10017000BA28F5014030850004308600F60A0830C0
:100180007606031DDA28FF30F600E3010C30750215
:10019000031CCC288617631406117308F700740833
:1001A000F8007508F9000C306318F902F908031912
:1001B000F9001C2983167608FA00031DE02802299D
:1001C000FA0BE3280229FA0BE628F128FA0BE928B2
:1001D0000729FA0BEC280729FA0B0C297718F428C1
:1001E000FB28771CF428FB28831276087C04860001
:1001F0007D0885001C29831276087E0486007F080E
:1002000085001C2977087618403E9B001029780845
:10021000761C403E9B00102979087618403E9B00D2
:100220001C141A088312E0000F39E10060067604FE
:0C02300086000513610885008C10090091
:02400E00503F21
:02420000770045
:02420200240096
:024204005d005b
:024206006d0049
:024208002e0086
:02420a006b0047
:02420c007b0035
:02420e00250089
:024210007f002d
:024212002f007b
:02421400770031
:02421600240082
:024218005d0047
:02421a006d0035
:02421c002e0072
:02421e006b0033
:024220007b0021
:02422200250075
:024224007f0019
:024226002f0067
:0242280077001d
:02422a0024006e
:02422c005d0033
:02422e006d0021
:024230002e005e
:024232006b001f
:024234007b000d
:02423600250061
:024238007f0005
:02423a002f0053
:02423c00770009
:02423e0024005a
:024240005d001f
:024242006d000d
:024244002e004a
:024246006b000b
:024248007b00f9
:02424a0025004d
:02424c007f00f1
:02424e002f003f
:024250007700f5
:02425200240046
:024254005d000b
:024256006d00f9
:024258002e0036
:02425a006b00f7
:02425c007b00e5
:02425e00250039
:024260007f00dd
:024262002f002b
:024264007700e1
:02426600240032
:024268005d00f7
:02426a006d00e5
:02426c002e0022
:02426e006b00e3
:024270007b00d1
:02427200250025
:024274007f00c9
:024276002f0017
:02427800130031
:02427a0013002f
:02427c0013002d
:02427e0013002b
:024280007700c5
:024282007700c3
:024284007700c1
:024286007700bf
:024288007700bd
:02428a007700bb
:02428c007700b9
:02428e007700b7
:024290007700b5
:024292007700b3
:02429400240004
:02429600240002
:02429800240000
:02429a002400fe
:02429c002400fc
:02429e002400fa
:0242a0002400f8
:0242a2002400f6
:0242a4002400f4
:0242a6002400f2
:0242a8005d00b7
:0242aa005d00b5
:0242ac005d00b3
:0242ae005d00b1
:0242b0005d00af
:0242b2005d00ad
:0242b4005d00ab
:0242b6005d00a9
:0242b8005d00a7
:0242ba005d00a5
:0242bc006d0093
:0242be006d0091
:0242c0006d008f
:0242c2006d008d
:0242c4006d008b
:0242c6006d0089
:0242c8006d0087
:0242ca006d0085
:0242cc006d0083
:0242ce006d0081
:0242d0002e00be
:0242d2002e00bc
:0242d4002e00ba
:0242d6002e00b8
:0242d8002e00b6
:0242da002e00b4
:0242dc002e00b2
:0242de002e00b0
:0242e0002e00ae
:0242e2002e00ac
:0242e4006b006d
:0242e6006b006b
:0242e8006b0069
:0242ea006b0067
:0242ec006b0065
:0242ee006b0063
:0242f0006b0061
:0242f2006b005f
:0242f4006b005d
:0242f6006b005b
:0242f8001300b1
:0242fa001300af
:0242fc001300ad
:0242fe001300ab
:00000001FF
